:1000000008308A00002800008A1D0A128A190A1680
:100010008A11831A0F28A500030EA6001428831244
:10002000A500030EA600A6140A08AD00A50E04083C
:10003000A7002008A8002108A9002208AA00230878
:10004000AB002408AC0083128B1D28280B184E2807
:100050000B1E2C288B1850288B1E30280B19522869
:100060008C308400001C36280C1854282708840083
:100070002808A0002908A1002A08A2002B08A30034
:100080002C08A4002D088A000A1A8A150A12260EC6
:1000900083008312250EA618831609008A11E3290E
:1000A0008A11692A8A112F298A11B0290710130889
:1000B00002309300831614185F2883125A28831283
:1000C00013085A08930083161418682883126328AB
:1000D000831213085B089300831614187128831287
:1000E0006C28831207140034071013088230930021
:1000F000831614187D28831278288312071400347D
:100100004130DA000230DB0056204230DA00DB01F9
:1001100056204530DA000830DB0056204630DA0041
:100120009830DB0056204730DA004408DB005620C8
:10013000D9014830DA005908DB0056204930DA008E
:100140004008DB0056204108D9004A30DA0059083F
:10015000DB0056204B30DA004708DB0056204C30DD
:10016000DA000130DB0056204D30DA000430DB00CD
:100170005620742000340710130881309300831632
:100180001418C4288312BF28831207140034313096
:10019000DA000830DB0056203230DA00DB0156206E
:1001A0003530DA000130DB0056203630DA006D30B1
:1001B000DB005620BB2000342E10C720BC01861265
:1001C000071505148515051505140630BD00AE1775
:1001D000003405152E118612071505148515AE116C
:1001E00000344130DA000230DB0056204230DA00C1
:1001F000DB0156204530DA000830DB00562046305F
:10020000DA009730DB0056204730DA002E08DB009A
:1002100056204830DA003008DB0056203108D9007B
:100220004930DA005908DB0056204A30DA00380835
:10023000DB0056203908D9004B30DA005908DB00C2
:1002400056204C30DA003408DB0056203508D9003F
:100250004D30DA005908DB00562074200034BE0B04
:100260008129BC0A0530BF000F30BE002E080F39AF
:10027000A0000F302002031D712940080319C1039B
:10028000C00339088039A300380800392304031D4E
:100290005B29C108031D50291E304002031980202C
:1002A00040084104031D5B292E088039A0008030DE
:1002B0002002031DDC2042080319C303C2034208C5
:1002C0004304031D702939084039A3003808003958
:1002D000230403196D2935176F293117E920712976
:1002E00031132E088039A00080302002031D81299F
:1002F000E920BD0B81290914AE10FF30BA0001308E
:10030000AE002F082E02031993292E08AF002E08E5
:100310000F39A0000F302002031D92290E30C100BA
:100320001030C000F12033083102031D9B29320830
:1003300030020319A0293108B3003008B200F120BF
:1003400037083502031DA829360834020319AD29E0
:100350003508B7003408B600F1200B118A11362891
:1003600010100030061A01300038031DD02901306A
:100370003B02031DD029C508031DCF29C408031D56
:10038000CF29B1162E12AE1239082039A300380831
:10039000003923040319CE29B516CF29E920D42921
:1003A0001730C500D430C40044080319C503C40382
:1003B000FF308F008C308E00101483164010831293
:1003C0000C108A1136280608C7002E080F39A00025
:1003D0000F302002031D182A0030061A0130D70002
:1003E0000030481A0130570600380319182A4812FD
:1003F000061A48160030061A01300038031D0D2A6F
:1004000001303B02031D0B2A2E16FF308F008C306B
:100410008E0010140C2AAE16182A10102E12AE12CE
:100420000E30C1001030C0001730C500D430C400F9
:100430002E080939A00009302002031D332A00309C
:10044000061B01300038031D332ABF0B332A39083D
:100450000839A3003808003923040319312AB515D7
:10046000332AB115E9200030861B01300038031D06
:10047000432A2E088039A000803020020319432A25
:100480000830BA00DC204708C8000B108A11362853
:10049000071013080330930083161418512A83128F
:1004A0004C2A8312130859089300831614185A2AE9
:1004B0008312552A83121308930183161418622A93
:1004C00083125D2A83121308DA0007145A08A10068
:1004D000003407101308A030930083161418722AF2
:1004E00083126D2A831213089301831614187A2A33
:1004F0008312752A83121308D90007145908A10022
:100500002108CB004B1C2E2B6630D9004822210835
:10051000CC00C3011E30C2004C08A0002008031903
:10052000C62A093020020319C82A80302002031984
:10053000CA2A013020020319D92A023020020319E5
:100540000B2B0330200203190B2B0530200203195B
:100550000B2B0430200203190B2B06302002031949
:100560000B2B0730200203190D2B08302002031932
:10057000182B0A3020020319222B0B3020020319FA
:10058000242B0C3020020319282B2E2BF1202E2B8C
:1005900080202E2BB901B8016830D90048222108EB
:1005A000B900B8016730D90048222108B804F12009
:1005B0002E2B31080039A300300810392304031909
:1005C000E32A3814341631080039A30030082039E2
:1005D00023040319ED2AB814B41631080039A30016
:1005E0003008403923040319F72A38153417310825
:1005F0000039A3003008803923040319012BB815F2
:10060000B417300831040319072B0730BA00B101C1
:10061000B001F1202E2BF1202E2B2E080339A00043
:1006200001302002031D162BB101B001F1202E2B49
:100630002E088039A000803020020319212BDC20F5
:10064000F1202E2BCE012E2B0130CE00F1202E2BAF
:100650000E30C1001030C000F1202E2BCB1CC22B5D
:100660007630D90048222108CD004D08A0009330F3
:1006700020020319542B9530200203197F2B94304C
:1006800020020319812B803020020319832B813033
:1006900020020319832B843020020319832B963008
:1006A00020020319872BC12BC3011E30C200013069
:1006B000BB007D30D9004822CA012108C9007C3026
:1006C000D9004822DA012108D9004908A300000115
:1006D000D90723080318013EDA0714305907C90067
:1006E00000300318013E5A07CA0064304907C400AD
:1006F00000300318013E4A07C5008020C22BBB0111
:10070000C22BBB01C22BC3011E30C200C22BC301CE
:100710001E30C20031080039A3003008103923040C
:100720000319942B3814341631080039A30030080B
:100730002039230403199E2BB814B416310800394C
:10074000A3003008403923040319A82B38153417A7
:1007500031080039A3003008803923040319B22B73
:10076000B815B4172E08023900380319BD2B07300D
:10077000CC000E30C1001030C000B101B001F1203A
:10078000C22BC22B2C30DA00DB0156208B108A11D1
:1007900036280F30DA009030DB000B088B13A500F1
:1007A000562025088B042A30DA00DB010B088B1356
:1007B000A500562025088B042930DA00D030DB0054
:1007C0000B088B13A500562025088B042830DA006F
:1007D0000230DB000B088B13A500562025088B0484
:1007E0003030DA000230DB000B088B13A5005620F6
:1007F00025088B044030DA000230DB000B088B1335
:10080000A500562025088B045030DA000230DB00AA
:100810000B088B13A500562025088B040D30DA0039
:10082000DB010B088B13A500562025088B046030D4
:10083000DA002030DB000B088B13A50056202508BA
:100840008B042030DA00FF30DB000B088B13A5008F
:10085000562025088B042130DA00E030DB000B083D
:100860008B13A500562025088B04DA011030DB001D
:100870000B088B13A500562025088B040130DA00E5
:10088000DB010B088B13A500562025088B040430D0
:10089000DA00DB010B088B13A500562025088B041A
:1008A0000530DA00DB010B088B13A5005620250864
:1008B0008B047030DA002230DB000B088B13A500AC
:1008C000562025088B042430DA00FF30DB000B08AB
:1008D0008B13A500562025088B042530DA00DB0198
:1008E0000B088B13A500562025088B040830DA006E
:1008F0000230DB000B088B13A500562025088B0463
:100900000930DA00DB010B088B13A50056202508FF
:100910008B040C30DA000F30DB000B088B13A500C2
:10092000562025088B042B30DA000330DB000B083F
:100930008B13A500562025088B040F30DA00DB014D
:100940000B088B13A500562025088B043130DA00E4
:100950000830DB000B088B13A500562025088B04FC
:100960003230DA002030DB000B088B13A500562054
:1009700025088B044130DA000230DB000B088B13B2
:10098000A500562025088B044230DA00DB010B0855
:100990008B13A500562025088B045130DA00023055
:1009A000DB000B088B13A500562025088B04523062
:1009B000DA00DB010B088B13A500562025088B04F9
:1009C0008A1555280030091901300038031DFB2C09
:1009D00039080039A3003808013923040319F22C1F
:1009E0003414FA2C0030091901300038031DFA2C98
:1009F0003014E920FE2C0030B105301000340030F6
:100A0000881A0130A00001302002031D1C2D390876
:100A10000239A3003808003923040319112DB51435
:100A20001B2D0030881A0130A00001302002031D68
:100A30001B2DB114E9201D2DB11000340030081B0E
:100A40000130A00001302002031D3B2D390801397F
:100A5000A3003808003923040319302D35143A2D2A
:100A60000030081B0130A00001302002031D3A2D88
:100A70003114E9203C2D31100034E224FF241E25DE
:100A80000034861207150910B101B0012E10AE1402
:100A9000BC01640008303A02031D5C2D2E08803929
:100AA000A0008030200203195B2D0B088B13A500DA
:100AB000DC2025088B047A2D05303C02031C692DAF
:100AC0003D25300831040319682D2E147A2D692D27
:100AD000792D0030081B0130A000013020020319DD
:100AE000492D0030881A0130A0000130200203197E
:100AF000492D2E1400340030881B01300038031DAE
:100B0000942D39080039A300380802392304031949
:100B10008B2DB414932D0030881B01300038031D39
:100B2000932DB014E920972D0030B105B01000349A
:100B3000BC01B101B0012E102E1505116400083062
:100B40003A02031DB12D2E088039A000803020020A
:100B50000319B02D0B088B13A500DC2025088B048E
:100B6000C72D02303C02031CC02D3D257B253008DB
:100B700031040319BF2DE9202E14C72DC02DC62D19
:100B80000030881B0130003803199E2D2E140034CC
:100B90000030071B01300038031DE12D39080039F2
:100BA000A3003808043923040319D82D3415E02D87
:100BB0000030071B01300038031DE02D3015E920FF
:100BC000E42D0030B105301100340030871B0130B6
:100BD0000038031DFE2D39080039A30038080839F4
:100BE00023040319F52DB415FD2D0030871B0130AA
:100BF0000038031DFD2DB015E920012E0030B10590
:100C0000B0110034C825E5250034003086190130C4
:100C1000A00001302002031D222E39080439A30050
:100C20003808003923040319172E3515212E0030FA
:100C300086190130A00001302002031D212E31153C
:100C4000E920232E31110034003006190130A000B4
:100C500001302002031D412E39081039A300380845
:100C6000003923040319362E3516402E003006199C
:100C70000130A00001302002031D402E3116E92072
:100C8000422E31120034052624260034BC01B10165
:100C9000B0012E10AE158612851007158511BC0106
:100CA000BC08031D632E08303A02031D612E2E146A
:100CB0000130AE000B088B13A500DC2025088B0447
:100CC000E72E6400502E0510640008303A02031D20
:100CD000772E2E088039A000803020020319762E4E
:100CE0000B088B13A500DC2025088B04E72E0130B0
:100CF0003C02031C8E2E3D250226300831040319C8
:100D00008D2E2E140130AE00BC0102303C020318BF
:100D10008B2E6400852EE72E8E2E9A2E0030071B18
:100D2000013000380319642E0030871B0130003871
:100D30000319642EBC01BC08031DB52E08303A020D
:100D4000031DB32E2E142E088039A00080302002FF
:100D50000319B22E0130AE000B088B13A500DC2066
:100D600025088B04E72E64009B2E8616BC01BC0868
:100D7000031DBC2E6400B72E07118514BC0164004E
:100D800008303A02031DD52E2E142E088039A000FB
:100D9000803020020319D42E0130AE000B088B13D3
:100DA000A500DC2025088B04E72E0A303C02031C3A
:100DB000E52E3D2502264326300831040319E42E92
:100DC000E9202E14E72EE52EE62EBF2E2E14003439
:100DD0008612071505148515AE118A1553290515B8
:100DE0002E118A15742905262426C825E5257B257C
:100DF000E224FF241E258A15EC295108A101500286
:100E00000318052F5008A000112FA0010830D200B0
:100E1000D00DA00D510820020318A000A10DD20B87
:100E2000082F8A15FA290030071B0130A000013075
:100E30002002031D272F39080039A3003808403944
:100E400023040319252F3417262F30172A2F00309B
:100E5000B10530130030871B0130A00001302002A3
:100E6000031D3E2F39080039A300380880392304B8
:100E700003193C2FB4173D2FB017412F0030B10597
:100E8000B0130030881B0130A00001302002031D88
:100E9000552F39080039A3003808203923040319D5
:100EA000532FB416542FB016582F0030B105B0127E
:100EB000003009190130A00001302002031D6C2F01
:100EC00039080039A30038081039230403196A2FA0
:100ED00034166B2F30166F2F0030B10530128A1583
:100EE000012AFF3FFF3FFF3FFF3FFF3FFF3FFF3F25
:100EF000FF3FFF3FFF3FFF3FFF3FFF3FFF3FFF3F02
:100F0000FF3FFF3FFF3FFF3FFF3FFF3FFF3FFF3FF1
:100F1000FF3FFF3FFF3FFF3FFF3FFF3FFF3FFF3FE1
:100F2000FF3FFF3FFF3FFF3FFF3FFF3FFF3FFF3FD1
:100F3000FF3FFF3FFF3FFF3FFF3FFF3FFF3FFF3FC1
:100F4000FF3FFF3FFF3FFF3FFF3FFF3FFF3FFF3FB1
:100F5000FF3FFF3FFF3FFF3FFF3FFF3FFF3FFF3FA1
:100F6000FF3FFF3FFF3FFF3FFF3FFF3FFF3FFF3F91
:100F7000FF3FFF3FFF3FFF3FFF3FFF3FFF3FFF3F81
:100F8000FF3FFF3FFF3FFF3FFF3FFF3FFF3FFF3F71
:100F9000FF3FFF3FFF3FFF3FFF3FFF3FFF3FFF3F61
:100FA000FF3FFF3FFF3FFF3FFF3FFF3FFF3FFF3F51
:100FB000FF3FFF3FFF3FFF3FFF3FFF3FFF3FFF3F41
:100FC000FF3FFF3FFF3FFF3FFF3FFF3FFF3FFF3F31
:100FD000FF3FFF3FFF3FFF3FFF3FFF3FFF3FFF3F21
:100FE000FF3FFF3FFF3FFF3FFF3FFF3FFF3FFF3F11
:100FF000FF3FFF3FFF3FFF3FFF3FFF3FFF3FFF3F01
:1010000084011F308305640085120130AE00013079
:10101000AF00B101B0018030B500B401FF30BA00BB
:10102000FF30CC008030B900B801FF308500FF30C0
:101030008600FF308700FF308800FF3089001030C5
:1010400083168500DF308600D0308700F8308800B6
:10105000063089000F308312BE00BC0181010730C9
:10106000A000A01D3B2807308101813084000008CA
:10107000C0390F3880006400813084000008C03916
:1010800020048000101035309000FF308F008C302D
:101090008E00813084000013831687120716871193
:1010A0003130831294008A11C92B8A15CF01BB01FC
:1010B0004812061A48168B168C30840000140B1642
:1010C0008B15C0308B04CE0164002E080339A000BC
:1010D00001302002031D79280030861801300038C5
:1010E000031D79281730C500D430C4008A1141256A
:1010F0008A152E080339A00003302002031DD128D1
:101100000030861801300038031DD128BC0104309E
:101110003C02031894280030861801300038031967
:1011200093280430BC00872800308618013000382E
:10113000031DD1282E080339A00003302002031913
:10114000A4288A1141258A152E080339A0000330EE
:101150002002031DD1282E080539A00005302002E9
:101160000319B5288A1198258A152E080539A0007B
:1011700005302002031DD1282E080939A0000930AE
:1011800020020319C6288A1146268A152E08093915
:10119000A00009302002031DD1280E30C1001030FC
:1011A000C0002E080939A00009302002031DDB28E9
:1011B0008A1143268A1502304C02FA3E031876291A
:1011C000063E042AFF30CC002E088039A000803073
:1011D0002002031922292E080339A000033020021F
:1011E0000319F5288A1141258A152E080339A00014
:1011F00003302002031D22292E080539A0000530E6
:101200002002031906298A1198258A152E08053906
:10121000A00005302002031D22292E080939A00054
:1012200009302002031917298A1146268A152E082B
:101230000939A00009302002031D22290E30C10007
:101240001030C0001730C5008430C4007629FF304C
:10125000CC002E080339A00001302002031D3329E1
:101260008A1141258A157629FF30CC002E080339D2
:10127000A00003302002031D4E292E080939A000CA
:101280000830200203194E292E080939A000093020
:10129000200203194E298A1146268A157629FF3025
:1012A000CC008A11E82E8A157629FF30CC002E0852
:1012B0000339A00003302002031D6F292E080539D1
:1012C000A0000430200203196F292E080539A00060
:1012D0000530200203196F298A1198258A1576296D
:1012E000FF30CC008A11EF2E8A15762907303A029A
:1012F000FF3E0318B729013E0E2AFF30BA002E0820
:101300000339A00003302002031989298A114125DD
:101310008A152E080339A00003302002031DB629C8
:101320002E080539A0000530200203199A298A11D8
:1013300098258A152E080539A00005302002031DC6
:10134000B6292E080939A000093020020319AB295B
:101350008A1146268A152E080939A0000930200274
:10136000031DB6290E30C1001030C000B7294F0848
:101370003C020319022A3C08CF00CE080319C829F1
:101380000B088B13A5008A11F1208A1525088B0400
:101390002E080339A00001302002031DD7290B08B5
:1013A0008B13A5008A11F1208A1525088B043008BB
:1013B00031040319E3290B088B13A5008A11F120CE
:1013C0008A1525088B042E080F39A0000F30200243
:1013D000031DED298A11F32E8A152E080339A0006A
:1013E00001302002031D022A3C08D0000A30D1003F
:1013F0008A11FD2E8A1509302002031D022A8A1146
:10140000132F8A15642863000A108A140A118207B0
:10141000272934294F2955297029E2280A108A14CE
:061420000A1182077D297C
:02400E00FE3F73
:00000001FF
